:020000040000FA
:06080000C3EF2FF012000F
:020806001200DE
:06080800E4EF05F0120010
:02080E00FEFFEB
:060818001CEF04F01200C9
:02081E000200D6
:100820000E080000F701000002000000E55F000074
:080830009901000052000000D4
:08083800D8CFE4FFE0CFE4FF9C
:10084000E46EDACFE4FFE2CFDAFFE9CFE4FFEACFEC
:10085000E4FFF6CFE4FFF7CFE4FFF5CFE4FFF3CFFB
:10086000E4FFF4CFE4FFFACFE4FF00EE1EF0140E35
:10087000E80403E3EECFE4FFFBD700EE32F00E0E08
:10088000E80403E3EECFE4FFFBD7E65236EC1BF0BF
:100890009EA200D19E92030E406E0E50EA6A510F46
:1008A000E96E010EEA22EF50405C30E10E50E96E35
:1008B000EA6AD890E936EA36690EE926010EEA229C
:1008C000EECF40F0EFCF41F041C040F0416A4050E0
:1008D000D76E0E50E96EEA6AD890E936EA36690EAC
:1008E000E926010EEA22EECF40F0EFCF41F0405072
:1008F000D66EF28AF294D58E0E50EA6A510FE96EE6
:10090000010EEA22040EEF6E0E50106E020E406EC3
:100910000F50EA6A510FE96E010EEA22EF50405C77
:1009200049E10F50E96EEA6AD890E936EA36690E75
:10093000E926010EEA22EE50ED1009E10F50EA6AB5
:10094000510FE96E010EEA22010EEF6E33D0080E50
:100950000F5C0CE2070E0F14406E010E405204E0D3
:10096000E846FE0B4006FCE189121AD0100E0F5C1F
:100970000CE2070E0F14406E010E405204E0E846F0
:10098000FE0B4006FCE18A120BD0070E0F14406EDE
:10099000010E405204E0E846FE0B4006FCE18B12DB
:1009A0000F50EA6A510FE96E010EEA22030EEF6E54
:1009B0000F500E6E0F2A060E0F5C02E1080E04D0D7
:1009C000130E0F5C03E1160E0F6E04D0180E0F5CB1
:1009D00001E10F6A000ED8800254000E03542EE28B
:1009E000112A000E12220250115C0350125826E305
:1009F000116A126A030E065C1FE20450EA6A480F8D
:100A0000E96E010EEA2280CFEFFF0450EA6A4B0F35
:100A1000E96E010EEA2281CFEFFF0450EA6A4E0F21
:100A2000E96E010EEA2282CFEFFF042A030E045C76
:100A300001E3046A062A02D0026A036A000ED88023
:100A40000754000E085419E20C50000816E2132A4D
:100A5000000E14220750135C085014580EE3136A5A
:100A6000146A030E0B5C07E2092A030E095C01E31A
:100A7000096A0B2A02D0076A086A0C5000080AE2C9
:100A8000156A1550040DF328C26E9E9C9F9C9D8C88
:100A9000C280C2829EAC2BD09E9CC450456E446ADC
:100AA000C35000014410426E45C043F01550060D7E
:100AB000F3CF40F0F4CF41F0000E4026010E41226A
:100AC0000950020D4050F324E96E4150F420EA6EC3
:100AD00042C0EEFF43C0EDFF152A0C50155C02E347
:100AE0009D9C05D01550040DF328C26EC282F2A45D
:100AF00042D0D59EF294F29A040E406E1050EA6AEB
:100B0000510FE96E010EEA22EF50405C34E1080E0D
:100B1000105C0DE2070E1014406E010E405204E00E
:100B2000E846FE0B4006FCE1E81C89161CD0100EBE
:100B3000105C0DE2070E1014406E010E405204E0EE
:100B4000E846FE0B4006FCE1E81C8A160CD0070EB6
:100B50001014406E010E405204E0E846FE0B4006C1
:100B6000FCE1E81C8B161050EA6A510FE96E010E89
:100B7000EA22020EEF6EE55200EE3FF00E0EE804A0
:100B800003E3E5CFEDFFFBD700EE31F0140EE804F0
:100B900003E3E5CFEDFFFBD7E5CFFAFFE5CFF4FFA9
:100BA000E5CFF3FFE5CFF5FFE5CFF7FFE5CFF6FFA4
:100BB000E5CFEAFFE5CFE9FFE5CFDAFFE550E5CF86
:100BC000E0FFE5CFD8FF1000DACFE4FFE652A1A2A4
:100BD0003FD0A1921D501DE01650B36E1750B26E5B
:100BE0001C2A1A501C5C34E31D6A0101991D8914EA
:100BF000896E9A1D8A148A6E9B1D8B148B6E9C1DA8
:100C00008C148C6E9D1D8D148D6E1850B36E195002
:100C10001DD01850B36E1950B26E1C2A1B501C5CAC
:100C200017E3010E1D6E010199518910896E9A51C9
:100C30008A108A6E9B518B108B6E9C518C108C6E1F
:100C40009D518D108D6E1650B36E1750B26E1C6A8A
:100C5000E552E5CFDAFF1100D9CFE6FFE1CFD9FFAA
:100C6000020EE126896A92680F0EC16EC2900C6A6C
:100C7000070EB46E8A6A93688B6A94688C6A95686A
:100C80008D6A96688B908B929490949294840201D2
:100C9000010ECD6F0101F769F8690A6A096A0B6AEA
:100CA000056A046A066A026A036A076A086A116AC0
:100CB000126A136A146A156ACA82CA80CA9CCA9ADE
:100CC000CA88CA96FA0ECB6EDF6ADFCF32F00C0EFE
:100CD000E76E3218E8AE02D0E73402D0E750325C5B
:100CE00036E2010EDB6ADBCF32F0030EE76E32181C
:100CF000E8AE02D0E73402D0E750325C26E2DFCF24
:100D000032F0336A32BE3368060E3302F3CF33F06B
:100D10003202F3CF32F0F4503326000E3226010EA9
:100D20003322010EDBCF34F0356A34BE3568D890FB
:100D30003436353632503424E96E33503520EA6E7D
:100D4000EE6AED6A010EDB2ACED7DF2ABED702019A
:100D5000C76BC86BC56BC66BC96BCA6BCB6BCC6BF7
:100D60000E6A0F6A106ADF6ADFCF32F0180EE76E84
:100D70003218E8AE02D0E73402D0E750325C1BE212
:100D8000DFCFE9FFEA6AE9BEEA68D890E936EA36D9
:100D9000690EE926010EEA22EE6AED6ADFCFE9FF6D
:100DA000EA6AE9BEEA68510EE926010EEA22010E5E
:100DB000EF6EDF2AD9D7D586D59AD59CF294F29AD0
:100DC000F194D08ECA949D829F92F28EF28CCA8446
:100DD000B190020EE15C02E2E16AE552E16EE55299
:100DE000E7CFD9FF1200D9CFE6FFE1CFD9FF050E3B
:100DF000E126020EDB6A030EDB6A040EDB6A3AECC4
:100E00001AF00650000809E221EC0DF0052A030E45
:100E1000055C01E1056A0606F4D70B50000809E2FB
:100E200051EC0DF00A2A030E0A5C01E10A6A0B0676
:100E3000F4D7200E0001E76E6019E8AE02D0E73467
:100E400002D0E750605D01E2EAD16D50020B01E093
:100E5000E6D1400EE66E400EE66E020EE66E45EC02
:100E60002AF0E552E552E552E76E030EE7CFDBFFCD
:100E7000DB50000801E369D1040EDB6A030EDB508E
:100E8000F36E040EDBCFF4FFF350F45C01E35DD1AD
:100E9000040EDB50EA6A400FE96E020EEA22EFCF41
:100EA000DFFF0101E65110E0E75100080DE2020109
:100EB000C751EA6A000FE96E070EEA22DFCFEFFFA3
:100EC000C72B0101E70731D1E25144E10D0E326E2B
:100ED000DF50325C05E00A0E336EDF50335C3AE1DE
:100EE000010EE26F0201C751EA6A000FE96E070EB8
:100EF000EA220D0EEF6EC72B010EDB6AC751F36EAF
:100F0000010EDBCFF4FFF350F45C1CE2010EDBCFEB
:100F1000E9FFEA6AE9BEEA68000EE926070EEA225E
:100F2000EF50E66E010EDBCFE9FFEA6AE9BEEA6840
:100F30009E0EE926010EEA22E552E750EF6E010E01
:100F4000DB2ADCD7F4D90101E66BE76B0201C76B42
:100F5000C86BEBD01B0EDF5C09E1DE5107E1010E2F
:100F6000DE6F1B0EDF6FE06BE16BDFD0DE050BE1A8
:100F70005B0EDF5C08E11B0EDF5D05E1E05103E184
:100F80005B0EE06FD2D0DE0566E1410EDF5C63E10F
:100F90001B0EDF5D60E15B0EE05D5DE1DF6BE06B32
:100FA000E16BDE6B010EDB6ADBCFE9FFEA6AE9BECB
:100FB000EA68000EE926070EEA22EF500D081CE051
:100FC000010EDBCFE9FFEA6AE9BEEA689E0EE92678
:100FD000010EEA22EF50E66E010EDBCFE9FFEA6A6E
:100FE000E9BEEA68000EE926070EEA22E552E7505C
:100FF000EF6E010EDB2AD8D7010EDBCFC7F202015C
:10100000C751EA6A000FE96E070EEA22EF6A270E5F
:10101000326E590E336E346A32C0E6FFE66E34C06B
:10102000E6FF51EC2EF0E552E552E552000EE66E79
:10103000070EE66E240E326E590E336E346A32C0DD
:10104000E6FFE66E34C0E6FF51EC2EF0356E050E7D
:10105000E15E35506AD0080EDF5C1CE10201C75129
:10106000000818E2C707C751EA6A000FE96E070EC9
:10107000EA22EF6A210E326E590E336E346A32C0A4
:10108000E6FFE66E34C0E6FF51EC2EF0E552E55285
:10109000E5524BD00D0EDF5C48E00A0EDF5C45E008
:1010A000200EDF5C42E30101DF6BE06BE16BDE6B86
:1010B0000201C751EA6A000FE96E070EEA22DFCF8C
:1010C000EFFF0101E26B0201C72B030EC75D0AE1CE
:1010D000420E0701005D06E1530E015D03E10101CF
:1010E000010EE66F0101E65120E0E7511EE1050E19
:1010F0000201C75D09E12C0E0701045D05E1300E18
:10110000035D0101E76F11D0060E0201C75D0DE11D
:101110002C0E0701055D09E1300E035D0A0DF3CFCA
:10112000E7F1300E045D0101E7270201C751326E7D
:10113000336A000E321806E1010E331803E10D8602
:10114000C76BC86B040EDB2A99D60D5067E00DA063
:101150000FD01B0E326E590E336E346A32C0E6FF6A
:10116000E66E34C0E6FF51EC2EF0E552E552E55252
:101170000DA40FD0FF0E326E580E336E346A32C09B
:10118000E6FFE66E34C0E6FF51EC2EF0E552E55284
:10119000E5520DA60FD0E30E326E580E336E346A50
:1011A00032C0E6FFE66E34C0E6FF51EC2EF0E552A9
:1011B000E552E5520DA80FD0C40E326E580E336EB4
:1011C000346A32C0E6FFE66E34C0E6FF51EC2EF022
:1011D000E552E552E5520DAC0FD0A30E326E580E1B
:1011E000336E346A32C0E6FFE66E34C0E6FF51EC7F
:1011F0002EF0E552E552E5520DAE0FD08A0E326E5A
:10120000580E336E346A32C0E6FFE66E34C0E6FF35
:1012100051EC2EF0E552E552E5520D6A3FD8050E2D
:10122000E15C02E2E16AE552E16EE552E7CFD9FF07
:101230001200D9CFE6FFE1CFD9FFE652C5C2DFFFEA
:10124000DF2A400E326EDF50325C01E1DF6A0201BC
:10125000C651DF5C01E122D80201C551EA6A000FE4
:10126000E96E020EEA22FE0EDBCFEFFFC52B400E29
:10127000C55D01E1C56BC651C55D01E10D84FE0E82
:10128000DBCF32F0336A32BE336832C0F3FF33C093
:10129000F4FFE552E552E7CFD9FF1200D9CFE6FFC0
:1012A000E1CFD9FFE6520201C551C65D3BE0020124
:1012B000D25103E043EC2BF0FAD70201C651D8809B
:1012C000C55517E2C651C55DDF6EDFCFE6FFC651DB
:1012D000336A000F326E020E332232C0E6FF33C093
:1012E000E6FFA5EC2AF0E552E552E552C5C2C6F28A
:1012F00017D0400ED880C655DF6EDFCFE6FFC6514F
:10130000336A000F326E020E332232C0E6FF33C062
:10131000E6FFA5EC2AF0E552E552E5520201C66B64
:1013200043EC2BF0E552E552E7CFD9FF1200D9CFBD
:10133000E6FFE1CFD9FF040EE126DE6ADD6A020E88
:10134000DB6A030EDB6A0201C851EA6A000FE96E2C
:10135000070EEA22EF50E66EE66A58EC2FF0E552EF
:10136000E552020EF3CFDBFF0201C82BC851326EEB
:10137000336A000E321804E1010E331801E1C86B24
:10138000020EDB50DE6EDD6AC851EA6A000FE96EBC
:10139000070EEA22EF502C0836E0C851EA6A000F27
:1013A000E96E070EEA22EF500D082DE0C851EA6AF7
:1013B000000FE96E070EEA22EF50E66EE66A58EC7F
:1013C0002FF0E552E552030EF3CFDBFF0201C82BED
:1013D000C851326E336A000E321804E1010E331820
:1013E00001E1C86B020EDBCF34F034C035F0346A53
:1013F000030EDB5000013424326E000E3520336EB4
:1014000032C0DEFFDD6E000EDFCF26F0010EDBCF37
:1014100027F0460E261801E1275001E1FED0490EC3
:10142000261802E1430E271801E1F4D0490E2618D0
:1014300002E1520E271801E1EAD0490E261802E116
:10144000530E271801E1E0D0530E261802E1430E97
:10145000271801E1D6D0530E261802E1520E2718A4
:1014600001E1CCD0530E261802E1530E271801E1FA
:10147000C2D0530E261802E1420E271801E1B8D05F
:10148000430E261802E1420E271801E1AED0430EAA
:10149000261802E1520E271801E1A4D04F0E26189B
:1014A00002E1420E271801E19AD0570E261802E1F8
:1014B0004D0E271801E191D0520E261802E14D0E73
:1014C000271801E188D0440E261802E1500E271893
:1014D00001E17FD04F0E261802E1500E271876E06A
:1014E000490E261802E1500E27186DE0580E2618F6
:1014F00002E1540E271864E0540E261801E127502B
:101500005DE0410E261801E1275056E0560E2618E0
:1015100001E127504FE0490E261801E1275048E02D
:101520004F0E261801E1275041E0550E261802E122
:10153000430E271839E0580E261802E1430E2718EB
:1015400030E0430E261801E1275029E0520E2618FC
:1015500001E1275022E0580E261802E1520E27180A
:1015600019E0030EDB505CE1020EDBCFE6FFE66A1A
:10157000DBCFE6FFE66A670E326E580E336E346AD2
:1015800032C0E6FFE66E34C0E6FF51EC2EF0356E59
:10159000070E64D0A2EC10F063D098D861D02DD99A
:1015A0005FD0A4EC10F05CD095D85AD0C1D958D0F7
:1015B00048DA56D066DA54D074DA52D0D3D850D044
:1015C000A0EC10F04DD014EC0FF04AD0B9EC0FF0B5
:1015D00047D044DB45D000DB43D0C0DA41D0C6EC75
:1015E00011F03ED0A6EC10F03BD059EC11F038D001
:1015F0001FEC13F035D0EFEC13F032D0F1EC13F018
:101600002FD0F3EC13F02CD0F5EC13F029D0F7EC3D
:1016100013F026D0F9EC13F023D0FBEC13F020D01C
:10162000030EDBCFE6FFE66A020EDBCFE6FFE66ADB
:10163000030EDBCFE6FFE66A020EDBCFE6FFE66ACB
:101640003F0E326E580E336E346A32C0E6FFE66EDD
:1016500034C0E6FF51EC2EF0356E0B0EE15E3550D6
:101660000201C851EA6A000FE96E070EEA22EF5044
:101670000D080DE00D500BE1520E326E336ADF5053
:10168000321803E1DE52DD50331801E00D8EC7C27F
:10169000C8F2040EE15C02E2E16AE552E16EE55255
:1016A000E7CFD9FF12000201CD510FE0440E326E98
:1016B0005F0E336E346A32C0E6FFE66E34C0E6FF7A
:1016C00051EC2EF0E552E552E55212002CEC06F0FA
:1016D00053EF0BF0D9CFE6FFE1CFD9FF030EE126A0
:1016E000E66AD9CFE6FFDACFE6FF010EE66ECFEC71
:1016F00017F0E552E552E552E552E66AD950010F7E
:10170000E66E000EDA20E66E020EE66ECFEC17F003
:10171000E552E552E552E5520D501AE1DF0417E1BA
:10172000D950010FE96EDACFEAFFEE50ED100AE072
:10173000010E326E336ADB50321808E1020EDB50C4
:10174000331804E1010EDBCFCDF201D00D8CABDFFD
:10175000030EE15C02E2E16AE552E16EE552E7CF99
:10176000D9FF1200D9CFE6FFE1CFD9FF030EE12662
:10177000020EDB6AE66A000EE66E000EE66E030EEF
:10178000E66ECFEC17F0E552E552E552E552E66A17
:10179000D950020FE66E000EDA20E66E010EE66EFC
:1017A000CFEC17F0E552E552E552E5520D501BE142
:1017B000020EDB500CE10050011003E1026A036AE3
:1017C00011D0CA8400C002F001C003F00BD0005059
:1017D000011003E1076A086A05D0CA8400C007F057
:1017E00001C008F060DF030EE15C02E2E16AE5524D
:1017F000E16EE552E7CFD9FF1200D9CFE6FFE1CF86
:10180000D9FF060EE126E66AD9CFE6FFDACFE6FF7A
:10181000010EE66ECFEC17F0E552E552E552E552C7
:10182000E66AD950010FE66E000EDA20E66E010E70
:10183000E66ECFEC17F0E552E552E552E552E66A66
:10184000D950020FE66E000EDA20E66E010EE66E4B
:10185000CFEC17F0E552E552E552E552E66AD95071
:10186000040FE66E000EDA20E66E010EE66ECFEC97
:1018700017F0E552E552E552E552E66AD950050FF8
:10188000E66E000EDA20E66E010EE66ECFEC17F083
:10189000E552E552E552E552E66AD950030FE66E8D
:1018A000000EDA20E66E010EE66ECFEC17F0E55280
:1018B000E552E552E5520D5031E1DF50926E010ED6
:1018C000DB50936E020EDB50946E040EDB50956E6F
:1018D000050EDB50966E030EDB500D0805E20D0E73
:1018E000F36E030EF3CFDBFF030EDB5005E10F0EAB
:1018F000C16EC2900C6A11D00C6AC26A030EDBCFB3
:10190000E6FF0F0EE552D880E754C16EBE0EC06EE2
:10191000C280030EDB500C6ECA84C5DE060EE15C8D
:1019200002E2E16AE552E16EE552E7CFD9FF12002B
:10193000D9CFE6FFE1CFD9FF020EE126E66AD9CF83
:10194000E6FFDACFE6FF010EE66ECFEC17F0E552C8
:10195000E552E552E552E76E010EE7CFDBFF0D5091
:1019600066E1010EDB5002E1DF50896E010EE66E8A
:10197000D9CFE6FFDACFE6FFE66ECFEC17F0E552FF
:10198000E552E552E552E76E010EE7CFDBFF0D5061
:101990004EE1010EDB5002E1DF508A6E010EE66E71
:1019A000D9CFE6FFDACFE6FFE66ECFEC17F0E552CF
:1019B000E552E552E552E76E010EE7CFDBFF0D5031
:1019C00036E1010EDB5002E1DF508B6E010EE66E58
:1019D000D9CFE6FFDACFE6FFE66ECFEC17F0E5529F
:1019E000E552E552E552E76E010EE7CFDBFF0D5001
:1019F0001EE1010EDB5002E1DF508C6E010EE66E3F
:101A0000D9CFE6FFDACFE6FFE66ECFEC17F0E5526E
:101A1000E552E552E552E76E010EE7CFDBFF0D50D0
:101A200006E1010EDB5002E1DF508D6E3CDE020E5E
:101A3000E15C02E2E16AE552E16EE552E7CFD9FFEF
:101A400012008450E66EE66A8350E66EE66A8250C3
:101A5000E66EE66A8150E66EE66A8050E66EE66AF9
:101A6000220E326E580E336E346A32C0E6FFE66ED6
:101A700034C0E6FF51EC2EF0356E0D0EE15E3550B0
:101A800012004C0E326E5F0E336E346A32C0E6FFC7
:101A9000E66E34C0E6FF51EC2EF0E552E552E55219
:101AA0001200D9CFE6FFE1CFD9FFE652DF6A200E60
:101AB000326E580E336E346A32C0E6FFE66E34C0C2
:101AC000E6FF51EC2EF0E552E552E552DF6A0C508C
:101AD000DF5C30E2DFCF32F0336A32BE3368060EAD
:101AE0003302F3CF33F03202F3CF32F0F450332627
:101AF000000E3226010E33220A50020D3250F3241A
:101B0000E96E3350F420EA6EEECFE6FFEFCFE6FF4A
:101B10001A0E346E580E356E366A34C0E6FFE66E25
:101B200036C0E6FF51EC2EF0376E050EE15E375001
:101B3000DF2ACDD7490E326E5F0E336E346A32C063
:101B4000E6FFE66E34C0E6FF51EC2EF0E552E552BA
:101B5000E552E552E552E7CFD9FF1200D9CFE6FFB3
:101B6000E1CFD9FF030EE126E66AD9CFE6FFDACF4F
:101B7000E6FFE66ECFEC17F0E552E552E552E5528E
:101B8000E66AD950020FE66E000EDA20E66E010E0C
:101B9000E66ECFEC17F0E552E552E552E5520D50F6
:101BA00011E1DECF32F0DDCF33F0000E325C100EEB
:101BB000335807E2DECFE9FFDDCFEAFF020EDBCFCD
:101BC000EFFF71DD030EE15C02E2E16AE552E16ED6
:101BD000E552E7CFD9FF1200D9CFE6FFE1CFD9FF19
:101BE000030EE126E66AD9CFE6FFDACFE6FFE66E1E
:101BF000CFEC17F0E552E552E552E5520D5024E1E5
:101C0000DECF32F0DDCF33F0000E325C100E3358F1
:101C100007E2DECFE9FFDDCFEAFF020EEFCFDBFF09
:101C2000020EDBCFE6FFE66A100E326E580E336E00
:101C3000346A32C0E6FFE66E34C0E6FF51EC2EF0A7
:101C4000356E050EE15E3550030EE15C02E2E16A9D
:101C5000E552E16EE552E7CFD9FF1200D9CFE6FF9A
:101C6000E1CFD9FF030EE126E66AD9CFE6FFDACF4E
:101C7000E6FF050EE66ECFEC17F0E552E552E552B1
:101C8000E552E66AD950010FE66E000EDA20E66EE4
:101C9000010EE66ECFEC17F0E552E552E552E55243
:101CA000E66AD950020FE66E000EDA20E66E010EEB
:101CB000E66ECFEC17F0E552E552E552E5520D50D5
:101CC00001E0A8D0020EDB50010801E2A0D0010E15
:101CD000DB50070801E29BD0410E326EDF50325CD0
:101CE0001AE1020EDB500CE1010EF36EDB5004E052
:101CF000D890F336E806FCE1F350F31C921689D035
:101D0000010EF36EDB5004E0D890F336E806FCE1F8
:101D1000F35092127ED0420E326EDF50325C1AE1E6
:101D2000020EDB500CE1010EF36EDB5004E0D890A4
:101D3000F336E806FCE1F350F31C93166AD0010E6B
:101D4000F36EDB5004E0D890F336E806FCE1F35084
:101D500093125FD0430E326EDF50325C1AE1020EF6
:101D6000DB500CE1010EF36EDB5004E0D890F3364B
:101D7000E806FCE1F350F31C94164BD0010EF36E11
:101D8000DB5004E0D890F336E806FCE1F3509412FF
:101D900040D0440E326EDF50325C1AE1020EDB504E
:101DA0000CE1010EF36EDB5004E0D890F336E80648
:101DB000FCE1F350F31C95162CD0010EF36EDB50B2
:101DC00004E0D890F336E806FCE1F350951221D0F8
:101DD000450E326EDF50325C1AE1020EDB500CE130
:101DE000010EF36EDB5004E0D890F336E806FCE118
:101DF000F350F31C96160DD0010EF36EDB5004E089
:101E0000D890F336E806FCE1F350961202D00D8C20
:101E100001D049DC030EE15C02E2E16AE552E16EC9
:101E2000E552E7CFD9FF1200D9CFE6FFE1CFD9FFC6
:101E3000030EE126020EDB6AE66AD9CFE6FFDACFAF
:101E4000E6FF050EE66ECFEC17F0E552E552E552DF
:101E5000E552E66AD950010FE66E000EDA20E66E12
:101E6000010EE66ECFEC17F0E552E552E552E55271
:101E70000D5075E1010EDB50070856E3410E326E3E
:101E8000DF50325C0BE1010EF36EDB5004E0D890C2
:101E9000F336E806FCE1F35080143FD0420E326E78
:101EA000DF50325C0BE1010EF36EDB5004E0D890A2
:101EB000F336E806FCE1F35081142FD0430E326E66
:101EC000DF50325C0BE1010EF36EDB5004E0D89082
:101ED000F336E806FCE1F35082141FD0440E326E54
:101EE000DF50325C0BE1010EF36EDB5004E0D89062
:101EF000F336E806FCE1F35083140FD0450E326E42
:101F0000DF50325C11E1010EF36EDB5004E0D8903B
:101F1000F336E806FCE1F3508414E76E020EE7CFD7
:101F2000DBFFDB5008E002D00D8C19D0010EF36E00
:101F3000020EF3CFDBFF020EDBCFE6FFE66A070EF1
:101F4000326E580E336E346A32C0E6FFE66E34C02D
:101F5000E6FF51EC2EF0356E050EE15E3550030EB6
:101F6000E15C02E2E16AE552E16EE552E7CFD9FFBA
:101F70001200D9CFE6FFE1CFD9FF030EE126E66AD2
:101F8000D9CFE6FFDACFE6FF050EE66ECFEC17F00D
:101F9000E552E552E552E552E66AD950010FE66E88
:101FA000000EDA20E66E010EE66ECFEC17F0E55279
:101FB000E552E552E552E66AD950020FE66E000E90
:101FC000DA20E66E010EE66ECFEC17F0E552E55230
:101FD000E552E5520D5001E0A9D0020EDB50010898
:101FE00001E2A0D0010EDB50070801E29BD0410EB8
:101FF000326EDF50325C1AE1020EDB500CE1010E52
:10200000F36EDB5004E0D890F336E806FCE1F350C1
:10201000F31C891689D0010EF36EDB5004E0D890D2
:10202000F336E806FCE1F35089127ED0420E326EA0
:10203000DF50325C1AE1020EDB500CE1010EF36E50
:10204000DB5004E0D890F336E806FCE1F350F31CD3
:102050008A166AD0010EF36EDB5004E0D890F33696
:10206000E806FCE1F3508A125FD0430E326EDF5077
:10207000325C1AE1020EDB500CE1010EF36EDB5014
:1020800004E0D890F336E806FCE1F350F31C8B161D
:102090004BD0010EF36EDB5004E0D890F336E80627
:1020A000FCE1F3508B1240D0440E326EDF50325CB4
:1020B0001AE1020EDB500CE1010EF36EDB5004E07E
:1020C000D890F336E806FCE1F350F31C8C162CD0C4
:1020D000010EF36EDB5004E0D890F336E806FCE125
:1020E000F3508C1221D0450E326EDF50325C1AE173
:1020F000020EDB500CE1010EF36EDB5004E0D890D1
:10210000F336E806FCE1F350F31C8D160DD0010EFA
:10211000F36EDB5004E0D890F336E806FCE1F350B0
:102120008D1202D00D8C02D053EC0BF0030EE15C4B
:1021300002E2E16AE552E16EE552E7CFD9FF120013
:1021400053EF0BF053EF0BF053EF0BF0D9CFE6FF4B
:10215000E1CFD9FF040EE126E66AD9CFE6FFDACF58
:10216000E6FF050EE66ECFEC17F0E552E552E552BC
:10217000E552E66AD950010FE66E000EDA20E66EEF
:10218000010EE66ECFEC17F0E552E552E552E5524E
:10219000E66AD950020FE66E000EDA20E66E030EF4
:1021A000E66ECFEC17F0E552E552E552E5520D50E0
:1021B00076E1D950020FE96EDACFEAFF720ED880CD
:1021C000EE542E0EED5441E3D950020FE96EDACFF2
:1021D000EAFFEE50ED101FE035683668376A2D0EC5
:1021E000E76E020EDBCF38F0030EDBCF39F0E7509D
:1021F0003826000E39223A6A3850355C326E395032
:102200003658336E3A503758346E020E32C0DBFF08
:10221000030E33C0DBFF010EDB50070816E3410E4F
:10222000326EDF50325C02E1DF6A11D0420E326E54
:10223000DF50325C02E1080E06D0430E326EDF50F2
:10224000325C03E1100EDF6E02D00D8C28D0010E3F
:10225000DB50DF24E96EEA6AD890E936EA36690E87
:10226000E926010EEA22020EDBCFEEFF030EDBCFE2
:10227000EDFF010EDB50DF24EA6A510FE96E010E1B
:10228000EA22EF040AE1010EDB50DF24EA6A510F73
:10229000E96E010EEA22020EEF6E53EC0BF0040E13
:1022A000E15C02E2E16AE552E16EE552E7CFD9FF77
:1022B0001200D9CFE6FFE1CFD9FF050EE126E66A8D
:1022C000D9CFE6FFDACFE6FF010EE66ECFEC17F0CE
:1022D000E552E552E552E552E66AD950020FE66E44
:1022E000000EDA20E66E010EE66ECFEC17F0E55236
:1022F000E552E552E552E66AD950030FE66E000E4C
:10230000DA20E66E010EE66ECFEC17F0E552E552EC
:10231000E552E552E66AD950010FE66E000EDA206A
:10232000E66E010EE66ECFEC17F0E552E552E5528F
:10233000E552E66AD950040FE66E000EDA20E66E2A
:10234000010EE66ECFEC17F0E552E552E552E5528C
:102350000D5012E1DFCFC0F2020EDBCFC2F2010E50
:10236000DBCFC1F2030EDBCFC3F2040EDBCFC4F22E
:10237000C0C289FF53EC0BF0050EE15C02E2E16A9A
:10238000E552E16EE552E7CFD9FF1200D9CFE6FF63
:10239000E1CFD9FF040EE126030EDB6A0201C8512A
:1023A000EA6A000FE96E070EEA22EF502C081DE0E2
:1023B0000201C851EA6A000FE96E070EEA22EF50E7
:1023C000E66EE66AE00E326E570E336E346A32C045
:1023D000E6FF33C0E6FF34C0E6FF51EC2EF0356E69
:1023E000050EE15E35500D8A20D10201C82B020195
:1023F000C851326E336A000E321802E1010E3318F2
:1024000002E10201C86BC0C289FF0201C11D89142B
:10241000326E891C0201C1153210E76E010EE7CF42
:10242000DBFF0201C851EA6A000FE96E070EEA22DB
:10243000EF500D0801E1F7D00201C851EA6A000F20
:10244000E96E070EEA22EF50E66EE66A58EC2FF0CE
:10245000E552E552020EF3CFDBFF300EF36E020EB3
:10246000DBCFF4FFF350F45C0FE3020EDB503908CE
:102470000BE3300E326E020EDBCFE7FF3250E75E29
:10248000020EE7CFDBFF19D0410EF36E020EDBCF59
:10249000F4FFF350F45C0FE3020EDB5046080BE34D
:1024A000370E326E020EDBCFE7FF3250E75E020ED0
:1024B000E7CFDBFF02D00D8CB8D0020EDB38F00B7B
:1024C000DF6E0201C82B0201C851326E336A000E62
:1024D000321802E1010E331802E10201C86B0D0E41
:1024E000326E0201C851EA6A000FE96E070EEA2255
:1024F000EF50325C02E10D8898D00201C851EA6ABF
:10250000000FE96E070EEA22EF50E66EE66A58EC1D
:102510002FF0E552E552020EF3CFDBFF300EF36EE3
:10252000020EDBCFF4FFF350F45C0FE3020EDB503E
:1025300039080BE3300E326E020EDBCFE7FF32506C
:10254000E75E020EE7CFDBFF19D0410EF36E020EFD
:10255000DBCFF4FFF350F45C0FE3020EDB504608D0
:102560000BE3370E326E020EDBCFE7FF3250E75E31
:10257000020EE7CFDBFF02D00D8C57D0020EDB50EE
:10258000DF24DF6E0201C82B0201C851326E336AAC
:10259000000E321802E1010E331802E10201C86B8D
:1025A000DF508A6E010EDB50896E0201C45105E0D6
:1025B000C4C2E6FFDFEC2FF0E552C0C289FF020182
:1025C000C35130E0030EC3C2DBFF0201C051020160
:1025D000C215326E0201C2518014325C0BE1030E4F
:1025E000DB5008E000000000000000000000030EC7
:1025F000DB06EBD7030EC3C2DBFF0201C0510201B1
:10260000C215326E0201C2518014325C0BE0030E1F
:10261000DB5008E000000000000000000000030E96
:10262000DB06EBD7FED653EC0BF0040EE15C02E2C6
:10263000E16AE552E16EE552E7CFD9FF1200D9CF4A
:10264000E6FFE1CFD9FF050EE126030EDB6A040E9B
:10265000DB6AE66AD950040FE66E000EDA20E66EF9
:10266000010EE66ECFEC17F0E552E552E552E55269
:10267000040EDB5004E0040EDB50380802E20D8C3F
:10268000A4D00201C851EA6A000FE96E070EEA22DF
:10269000EF502C081DE00201C851EA6A000FE96EF4
:1026A000070EEA22EF50E66EE66AE00E326E570E33
:1026B000336E346A32C0E6FF33C0E6FF34C0E6FF53
:1026C00051EC2EF0356E050EE15E35500D8A7DD051
:1026D0000201C82B0201C851326E336A000E321853
:1026E00002E1010E331802E10201C86BC0C289FF8A
:1026F0000201C11D8914326E891C0201C1153210FC
:10270000E76E010EE7CFDBFF040EDB505CE0020159
:10271000C851EA6A000FE96E070EEA22EFCFDFFF29
:102720000201C82B0201C851326E336A000E321802
:1027300002E1010E331802E10201C86B040EDB0650
:10274000DF508A6E010EDB50896E0201C45105E034
:10275000C4C2E6FFDFEC2FF0E552C0C289FF0201E0
:10276000C35130E0030EC3C2DBFF0201C0510201BE
:10277000C215326E0201C2518014325C0BE1030EAD
:10278000DB5008E000000000000000000000030E25
:10279000DB06EBD7030EC3C2DBFF0201C05102010F
:1027A000C215326E0201C2518014325C0BE0030E7E
:1027B000DB5008E000000000000000000000030EF5
:1027C000DB06EBD7A1D753EC0BF0050EE15C02E280
:1027D000E16AE552E16EE552E7CFD9FF120053EF0F
:1027E0000BF053EF0BF053EF0BF053EF0BF053EFF5
:1027F0000BF053EF0BF0D9CFE6FFE1CFD9FF0F0E6F
:10280000E126320EF36E0C0EF3CFDBFF010EF36EFA
:102810000D0EF3CFDBFF010EF36E0E0EF3CFDBFFD9
:10282000E66AD950080FE66E000EDA20E66E030E57
:10283000E66EB5DBE552E552E552E552D950080F98
:10284000E96EDACFEAFFEE50ED1012E1010EE66E0E
:10285000D9500A0FE66E000EDA20E66E050EE66E1F
:102860009EDBE552E552E552E552010EE66E0FD0D1
:10287000E66AD9500A0FE66E000EDA20E66E050E03
:10288000E66E8DDBE552E552E552E552E66AD95037
:102890000B0FE66E000EDA20E66E010EE66E7FDBB1
:1028A000E552E552E552E552010EE66ED9500C0FA5
:1028B000E66E000EDA20E66E010EE66E70DBE55283
:1028C000E552E552E5520D5001E05FD3D950080FB3
:1028D000E96EDACFEAFFEE50ED104FE1B190A09231
:1028E000410E0201D05D0CE1010ECFC2E7FFE752BD
:1028F00004E0E846FE0BE706FCE1E81C891643D33A
:10290000420ED05D0CE1010ECFC2E7FFE75204E0BA
:10291000E846FE0BE706FCE1E81C8A1634D3430EBA
:10292000D05D0CE1010ECFC2E7FFE75204E0E846BC
:10293000FE0BE706FCE1E81C8B1625D3440ED05DA8
:102940000CE1010ECFC2E7FFE75204E0E846FE0BC0
:10295000E706FCE1E81C8C1616D3450ED05D01E0BD
:1029600012D3010ECFC2E7FFE75204E0E846FE0BA8
:10297000E706FCE1E81C8D1606D3080EDBCF36F027
:10298000090EDBCF37F0386A396A640E296E2A6A7D
:102990002B6A2C6A36C024F037C025F038C026F0E8
:1029A00039C027F020EC2FF020C036F021C037F0DE
:1029B00022C038F023C039F00C0EDBCF32F0336A7E
:1029C000346A356A296A1B0E2A6EB70E2B6E2C6A82
:1029D00032C024F033C025F034C026F035C027F0D3
:1029E00020EC2FF020C032F021C033F022C034F0B0
:1029F00023C035F020C024F021C025F022C026F0ED
:102A000023C027F036C029F037C02AF038C02BF099
:102A100039C02CF09AEC2CF024C0DEFF25C0DEFF7C
:102A200026C0DEFF27C0DDFFDD52DD52080EDBCF02
:102A300036F0090EDBCF37F0386A396A640E296E3A
:102A40002A6A2B6A2C6A36C024F037C025F038C0B9
:102A500026F039C027F020EC2FF020C036F021C03E
:102A600037F022C038F023C039F00C0EDBCFE6FF80
:102A7000640EE552D880E754326E336A346A356AA0
:102A8000296A1B0E2A6EB70E2B6E2C6A32C024F0F8
:102A900033C025F034C026F035C027F020EC2FF0ED
:102AA00020C032F021C033F022C034F023C035F012
:102AB00020C024F021C025F022C026F023C027F03A
:102AC00036C029F037C02AF038C02BF039C02CF0BE
:102AD0009AEC2CF0040E24C0DBFF050E25C0DBFFB2
:102AE000060E26C0DBFF070E27C0DBFFD9CFE9FFAC
:102AF000DACFEAFFD880FF0EEE54FF0EEE54000E40
:102B0000EE54000EEE5423E2800EF36E0D0EF3CF62
:102B1000DBFFD9CFE9FFDACFEAFFEECF24F0EECF2B
:102B200025F0EECF26F0EFCF27F0800E296E2A6A2F
:102B30002B6A2C6A7EEC2FF024C0DEFF25C0DEFF5E
:102B400026C0DEFF27C0DDFFDD52DD5205D0010EBD
:102B5000F36E0D0EF3CFDBFFD9CFE9FFDACFEAFF3B
:102B6000280EEE5C000EEE58000EEE58000EEE58E9
:102B700007E2280EDE6EDE6ADE6ADD6ADD52DD52B5
:102B8000D950040FE96EDACFEAFFD880FF0EEE5479
:102B9000FF0EEE54000EEE54000EEE5425E2800EB1
:102BA000F36E0E0EF3CFDBFF040EDBCF24F0050E29
:102BB000DBCF25F0060EDBCF26F0070EDBCF27F0AC
:102BC000800E296E2A6A2B6A2C6A7EEC2FF0040E86
:102BD00024C0DBFF050E25C0DBFF060E26C0DBFF91
:102BE000070E27C0DBFF05D0010EF36E0E0EF3CFEC
:102BF000DBFFD950040FE96EDACFEAFF280EEE5C56
:102C0000000EEE58000EEE58000EEE580BE2280EA5
:102C1000F36E040EF3CFDBFF050EDB6A060EDB6AF4
:102C2000070EDB6A040EDBCF32F0050EDBCF33F08C
:102C3000060EDBCF34F0070EDBCF35F0140E325E1C
:102C4000000E335A345A355A040E32C0DBFF050EDB
:102C500033C0DBFF060E34C0DBFF070E35C0DBFFE1
:102C6000D9CFE9FFDACFEAFFEECF32F0EECF33F083
:102C7000EECF34F0EFCF35F0140E325E000E335A43
:102C8000345A355A32C0DFFF010E33C0DBFF020E6B
:102C900034C0DBFF030E35C0DBFF0B0EDB50070833
:102CA00001E2D6D0000EF36E0C0EDBCFF4FFF35032
:102CB000F45C01E2CDD00C0EDB50630801E2C8D019
:102CC000B1B0A9D00101996B9A6B9B6B9C6B9D6B0A
:102CD000410E326E0A0EDB50325C19E1010EF36ECA
:102CE0000B0EDB5004E0D890F336E806FCE1F3501D
:102CF000F31C9216010EF36E0B0EDB5004E0D8901D
:102D0000F336E806FCE1F350010199137BD0420E43
:102D1000326E0A0EDB50325C19E1010EF36E0B0EBF
:102D2000DB5004E0D890F336E806FCE1F350F31CE6
:102D30009316010EF36E0B0EDB5004E0D890F336C1
:102D4000E806FCE1F35001019A135CD0430E326EA9
:102D50000A0EDB50325C19E1010EF36E0B0EDB50F4
:102D600004E0D890F336E806FCE1F350F31C941627
:102D7000010EF36E0B0EDB5004E0D890F336E8063C
:102D8000FCE1F35001019B133DD0440E326E0A0E5C
:102D9000DB50325C19E1010EF36E0B0EDB5004E0E8
:102DA000D890F336E806FCE1F350F31C9516010EBB
:102DB000F36E0B0EDB5004E0D890F336E806FCE12E
:102DC000F35001019C131ED0450E326E0A0EDB50EB
:102DD000325C3EE1010EF36E0B0EDB5004E0D89046
:102DE000F336E806FCE1F350F31C9616010EF36E81
:102DF0000B0EDB5004E0D890F336E806FCE1F3500C
:102E000001019D130B0EDBCFCFF20A0EDBCFD0F208
:102E1000010E1D6E1C6AD9CFE9FFDACFEAFFD88018
:102E2000FF0EEE54FF0EEE54000EEE54000EEE5464
:102E30000FE3D950040FE96EDACFEAFFD880FF0E16
:102E4000EE54FF0EEE54000EEE54000EEE5402E26D
:102E50000D8C9BD036683768386A396AD9CFE9FF5C
:102E6000DACFEAFFEE50365C326EEE503758336EF2
:102E7000EE503858346EEE503958356E32C0DFFFA0
:102E8000010E33C0DBFF020E34C0DBFF030E35C082
:102E9000DBFF36683768386A396AD950040FE96E43
:102EA000DACFEAFFEE50365C326EEE503758336EB2
:102EB000EE503858346EEE503958356E040E32C02C
:102EC000DBFF050E33C0DBFF060E34C0DBFF070E51
:102ED00035C0DBFFF29ED9CFE9FFDACFEAFFEECFB4
:102EE00032F0EECF33F0EECF34F0EFCF35F0080E06
:102EF000D8903532343233323232E806F9E132508A
:102F0000166ED9CFE9FFDACFEAFFEECF32F0EECF7F
:102F100033F0EECF34F0EFCF35F03250176E040EB1
:102F2000DBCF32F0050EDBCF33F0060EDBCF34F013
:102F3000070EDBCF35F0080ED890353234323332FD
:102F40003232E806F9E13250186E040EDBCF32F06F
:102F5000050EDBCF33F0060EDBCF34F0070EDBCFF0
:102F600035F03250196E0D0EDB501A6E0E0EDB501E
:102F70001B6EF28EB1B007D0B192B198B19AA28215
:102F8000A192A082B18053EC0BF00F0EE15C02E243
:102F9000E16AE552E16EE552E7CFD9FF1200D9CFE1
:102FA000E6FFE1CFD9FF040EE126030EDB6A0D0E2A
:102FB000326E0201C851EA6A000FE96E070EEA227A
:102FC000EF50325C05E1FB0EDB5044E10D8842D04E
:102FD000C851EA6A000FE96E070EEA22EF502C088A
:102FE0001FE0FB0EDB501AE1C851EA6A000FE96EE0
:102FF000070EEA22EF50E66EE66AE00E326E570EDA
:10300000336E346A32C0E6FFE66E34C0E6FF51EC40
:103010002EF0356E050EE15E35500D8A020E90D110
:10302000C82BC851326E336A000E321804E1010E0B
:10303000331801E1C86B0D0E326EC851EA6A000FF9
:10304000E96E070EEA22EF50325C06E1FB0EDB5020
:1030500001E10D88030E74D12D0E326EC851EA6A5B
:10306000000FE96E070EEA22EF50325C27E1040EF2
:10307000336EFE0EDB50335C21E0050E346EFE0E27
:10308000DB50345C1BE0FE0EDB0401E12FD1030EAC
:10309000326EFE0EDB50325C01E128D1010EF36E80
:1030A000030EF3CFDBFFC82BC851326E336A000E1C
:1030B000321804E1010E331801E1C86B040E326EC0
:1030C000FE0EDB50325C11E0050E336EFE0EDB505F
:1030D000335C0BE0050EE66ED9CFE6FFDACFE6FFF4
:1030E0003BD9E552E552E5523DD0C851EA6A000F9E
:1030F000E96E070EEA22EFCF32F0336A346A32C04B
:10310000DFFF010E33C0DBFF020E34C0DBFF050E14
:10311000326EFE0EDB50325C19E1000EDFCFE6FFAF
:10312000010EDBCFE6FF58EC2FF0E552E552F3CF6E
:1031300032F0F4CF33F0346A33BE346832C0DFFF8C
:10314000010E33C0DBFF020E34C0DBFF0201C82BCF
:10315000C851326E336A000E321804E1010E331882
:1031600001E1C86B030EDB501DE0DFCF32F0010E32
:10317000DBCF33F0020EDBCF34F02A682B682C68EB
:1031800032C025F033C026F034C027F0CEEC2CF04E
:1031900022C032F022C0DFFF010E23C0DBFF020E8F
:1031A00024C0DBFFFE0EDB5026E1DFCF32F0010E44
:1031B000DBCF33F0020EDBCF34F03434000E3418A2
:1031C00007E6D8807F0E3254000E3354000E34547C
:1031D00001E28CD0D9CFE9FFDACFEAFF020ED88026
:1031E000EB50FF0A06E6800EEE5CFF0EEE58FF0E77
:1031F000EF5801E27BD0FE0EDB0424E1DFCF35F097
:10320000010EDBCF36F0020EDBCF37F03734000E85
:10321000371807E6D880FF0E3554000E3654000EDE
:10322000375464E3D9CFE9FFDACFEAFF020ED89032
:10323000EB50000A06E6000EEE5C000EEE58000EA3
:10324000EF5854E3020E386EFE0EDB50385C24E17A
:10325000DFCF39F0010EDBCF3AF0020EDBCF3BF0CF
:103260003B34000E3B1807E6D880FF0E39547F0E22
:103270003A54000E3B543AE3D9CFE9FFDACFEAFFE4
:10328000020ED880EB50FF0A06E6000EEE5C800EC0
:10329000EE58FF0EEF582AE3030E3C6EFE0EDB5095
:1032A0003C5C27E1DFCF3DF0010EDBCF3EF0020EAC
:1032B000DBCF3FF03F34000E3F1807E6D880FF0E0B
:1032C0003D54FF0E3E54000E3F5410E3D9CFE9FFAA
:1032D000DACFEAFF020ED890EB50000A06E6000EA5
:1032E000EE5C000EEE58000EEF5803E20D8C010E5E
:1032F00027D0FE0EDB50030A16E0010A14E0030A91
:1033000008E0050A06E0010A04E0050A02E0040EEE
:1033100017D0FC0EDBCFE9FFFD0EDBCFEAFF000E7E
:10332000DFCFEFFF0CD0FC0EDBCFE9FFFD0EDBCFD4
:10333000EAFF000EDFCFEEFF010EDBCFEDFF000E48
:10334000326E040EE15C02E2E16AE552E16E325057
:10335000E552E7CFD9FF1200D9CFE6FFE1CFD9FF81
:10336000020EE126FD0EDBCFE9FFFE0EDBCFEAFF0A
:10337000EE6AEE6AEE6A010EDB6AFC0EDB50F36E5B
:10338000010EDBCFF4FFF350F45C53E20201C851AD
:10339000EA6A000FE96E070EEA22EFCFDFFF300E78
:1033A000DF5C42E3DF5039083FE3FD0EDBCFE9FF8E
:1033B000FE0EDBCFEAFFEECF35F0EECF36F0EFCFEB
:1033C00037F00A0E2A6E2B6A2C6A35C025F036C0FB
:1033D00026F037C027F0CEEC2CF0300EDF5C386ED4
:1033E000396A3A6A22503824326E23503920336EBB
:1033F00024503A20346EFD0EDBCFE9FFFE0EDBCF0A
:10340000EAFF32C0EEFF33C0EEFF34C0EEFF020130
:10341000C82BC851326E336A000E321807E1010E14
:10342000331804E1C86B02D0000E04D0010EDB2A71
:10343000A4D7010E326E020EE15C02E2E16AE552AF
:10344000E16E3250E552E7CFD9FF12000650E66E2A
:10345000E66AD40E326E570E336E346A32C0E6FF1F
:10346000E66E34C0E6FF51EC2EF0356E050EE15EDF
:10347000355012000001605108E0010E326E6D50AF
:10348000020B01E0010E325C1BE10101E807000EB6
:10349000E95BEA510BE1E851E91111E18B80D00EB3
:1034A000E86F070EE96F010EEA6F1200E851E911AB
:1034B0004DE18B90D00EE86F070EE96FEA6B1200BA
:1034C000600509E0020E605D06E0040E605D03E049
:1034D000100E605D02E18B801200200E605D36E10F
:1034E0000101E807000EE95BEA510AE1E851E91140
:1034F0002DE18B80100EE86F270EE96F010E18D0BA
:10350000EA050AE1E851E91121E18B90100EE86F1C
:10351000270EE96F020E0CD0020EEA5D0BE1E851B6
:10352000E91114E18B80A00EE86F860EE96F030E9F
:10353000EA6F1200030EEA5D09E3E851E91106E1C2
:103540008B90100EE86F270EE96FEA6B120082A4D1
:04355000010C000C5E
:0C355400D9CFE6FFE1CFD9FFE652A09AE4
:103560006A6A686A706A030EE66EE66AE66A710E57
:10357000E66E0F0EE66E04EC2EF0326E050EE15E86
:103580003250160E6F6E9F0E6B6E7B0E696EDF6A89
:10359000DF50326E336A100E325C000E335810E288
:1035A000DF50040DF3CFE9FFF4CFEAFF000EE92668
:1035B000040EEA22EE6AEE6AEE6AEE6ADF2AE8D7C5
:1035C0006D8C6E6A6D986D9C68A607D06896000138
:1035D0007B6B806B816B826BF7D70001010E966F5E
:1035E000976F986B996B886BDF6A040EDF5C26E23D
:1035F000EA6ADF34FE0BEA36E96E6F0EE926000E4A
:10360000EA22EE6AED6AEA6ADF34FE0BEA36E96E18
:10361000670EE926000EEA22EE6AED6ADF50EA6ADA
:103620008C0FE96E000EEA22EF6ADF50EA6A900F13
:10363000E96E000EEA22EF6ADF2AD7D70001080EF2
:103640006F6F040E706F160E706E0401400E026FE5
:10365000040E036F400E016F840E006F0001616B5A
:10366000606BE552E552E7CFD9FF1200D9CFE6FFF4
:10367000E1CFD9FFE6520001600507E16DBA05D040
:10368000686A69806988020E606F6850040B05E003
:103690006950040B02E06894BFD86DB250D06850F6
:1036A000010B09E06950010B06E054DFA08A00011C
:1036B000040E606F68906850100B05E06950100BA5
:1036C00002E095D8689868AC12D069AC0FD0010EB2
:1036D000E66EE66A000EE66EE66A730EE66EE66A6F
:1036E0006AEC2DF0326E060EE15E3250689C685036
:1036F000200B04E06950200B01E060D86850020BF9
:1037000013E06950020B10E0010EE66EE66A000E4F
:10371000E66EE66AE6687F0EE66E6AEC2DF0326EC3
:10372000060EE15E32506A6A040E0001E76E60190F
:10373000E8AE02D0E73402D0E750605D02E2A19A21
:1037400038D069A635D0DF6A040EDF5C31E268A6A6
:103750002FD06CCF89F000018951780BE842E84204
:10376000E8428A6F689689B506D08A51EA6A900F56
:10377000E96E000E05D08A51EA6A8C0FE96E000EE0
:10378000EA22EF708A5102E15ED810D0000EE66E98
:10379000E66A890EE66E000EE66E720EE66EE66A68
:1037A0006AEC2DF0326E060EE15E3250DF2ACCD785
:1037B000A19AE552E552E7CFD9FF120070A015D0CB
:1037C00063C0E9FF64C0EAFFEF5080080DE16FC0FD
:1037D000E9FF70C0EAFFEF50840806E163C0E9FF2B
:1037E00064C0EAFF8C0EEF6E7090689A12006984D4
:1037F00068986D820001010E886F000EE66EE66A21
:10380000E66EE66A750EE66EE66A6AEC2DF0326EDA
:10381000060EE15E325012000001886B000EE66E6B
:10382000E66AE66EE66A740EE66EE66A6AEC2DF00B
:10383000326E060EE15E32506D92699468A402D039
:103840006894FCD71200D9CFE6FFE1CFD9FFE6524A
:10385000FD0E0001891553E17E0E8915E8407F0BAE
:10386000040DF3CF63F0F4CF64F0000E6327040E71
:10387000642363C065F064C066F0657563C0E9FFEA
:1038800064C0EAFFEF503C0BE842E8420D0835E126
:10389000DF6A080EDF5C23E263C0E9FF64C0EAFF71
:1038A000020EE926000EEA22EE50EFCFEAFFE96EA3
:1038B000EF50E66EDF50EA6A400FE96E040EEA222E
:1038C000E552E750EF6E63C0E9FF64C0EAFF020E05
:1038D000E926000EEA22EE2AEF22DF2ADAD763C0B9
:1038E000E9FF64C0EAFF020EE926000EEA22400E5C
:1038F000EE6E040EED6E0DD807D03AD805D0FD0E51
:103900008915040801E159D8E552E552E7CFD9FFFE
:1039100012000001776B956B986B996B8B6B786BD2
:103920006FC0E9FF70C0EAFFEF9E6F756FC0E9FFDF
:1039300070C0EAFFEF9E6F7565C0E9FF66C0EAFFE1
:10394000EF9E7B6B7C6B7D6B806B816B826B8CD80D
:10395000000EE66EE66AE66EE66A030EE66EE66A5C
:103960006AEC2DF0326E060EE15E325003EF20F06D
:10397000020E0001785D02E1C3EF20F0786B8B51FD
:103980001AE165C0E9FF66C0EAFFEE52400EEF6E35
:1039900065C0E9FF66C0EAFF020EE926000EEA22D2
:1039A000400EEE6E040EED6E65C0E9FF66C0EAFFE4
:1039B0008C0EEF6E12008B6B1200D9CFE6FFE1CFB9
:1039C000D9FFE6526FC0E9FF70C0EAFFEF50400B2D
:1039D00001E0010EDF6E00016F75080E605D08E109
:1039E00042C46EFF6E5002E0100E01D0040E606FF4
:1039F000780526E16FC0E9FF70C0EAFF020EE926F4
:103A0000000EEA22480EEE6E040EED6E5DDB020E35
:103A10000001775D06E16FC0E9FF70C0EAFF840E28
:103A20000DD0DF5006E16FC0E9FF70C0EAFFC80E9D
:103A300005D06FC0E9FF70C0EAFF880EEF6E0FD0AF
:103A400080AF0CD08351841107E005D084C0FAFF09
:103A500000018351F96EFADF0001809F786BE55217
:103A6000E552E7CFD9FF120004014051600BE84254
:103A7000E842E842E842E842000901E01200415110
:103A80000C0A50E00B0A3FE00C0A31E0010A22E088
:103A90000B0A1EE0020A1CE0030A18E0080A10E004
:103AA000010A0CE00F0A08E0030A01E0120000011D
:103AB0007B8F080E606F12004CEF1FF062EF21F059
:103AC0000001610E796F000E7A6F0CD0A9EF1FF024
:103AD00093EF1DF044510001796F7A6B620E7927E4
:103AE000000E7A237B81010E7C6F7B8F1200000118
:103AF0007B8F04014451EA6A620FE96E000EEA22EC
:103B000042C4EFFF1200000EE66EE66AE66EE66A59
:103B1000020EE66EE66A6AEC2DF0326E060EE15E8B
:103B2000325012001200D9CFE6FFE1CFD9FF030EC9
:103B3000E1260401420510E140511F0B00090CE190
:103B400000017B8F030E0401415D04E10001010EC1
:103B5000876F02D00001876B0401425101E003D15D
:103B600040511F0B020801E0FED044510F0B000929
:103B700001E1F9D044510F0B030801E2F4D0200E0B
:103B80000001605D01E0EFD07B8F040144BF16D0DF
:103B900044510F0BE96EEA6AD890E936EA36670EAF
:103BA000E926000EEA22EECFDEFFEDCFDDFF445125
:103BB0000F0BEA6A900FE96E000E15D044510F0BFF
:103BC000E96EEA6AD890E936EA366F0EE926000E09
:103BD000EA22EECFDEFFEDCFDDFF44510F0BEA6AA4
:103BE0008C0FE96E000EEA22020EEFCFDBFFD950F8
:103BF000020FE96EDACFEAFFEF50010B03E1000E8E
:103C0000DF9401D0DF8444BF0BD044510F0BE96E29
:103C1000EA6AD890E936EA36670EE926000E0AD03D
:103C200044510F0BE96EEA6AD890E936EA366F0E16
:103C3000E926000EEA22DECFEEFFDDCFEDFF030E18
:103C4000415D20E1DECFE9FFDDCFEAFFEF50800BE1
:103C500011E044BF07D044510F0BEA6A900FE96EA0
:103C6000000E06D044510F0BEA6A8C0FE96E000E6D
:103C7000EA22EF82840EDECFE9FFDDCFEAFFE850D3
:103C8000EF1271D0DF74DECFE9FFDDCFEAFFEF5036
:103C9000800B1BE0DECFE9FFDDCFEAFFEF9EDECF3A
:103CA000E9FFDDCFEAFFEF8C020EE66EE66ADECFBB
:103CB000E6FFDDCFE6FF050EE66EE66A6AEC2DF064
:103CC000326E060EE15E325005D0DECFE9FFDDCF69
:103CD000EAFFEF8CDF74D950020FE96EDACFEAFF0A
:103CE000EF50020B0EE1DECFE9FFDDCFEAFFEF5030
:103CF000800B32E0DECFE9FFDDCFEAFFEF50040BAF
:103D00002BE1040144BF07D044510F0BEA6A900F26
:103D1000E96E000E06D044510F0BEA6A8C0FE96E73
:103D2000000EEA22EF923B0E326EDECFE9FFDDCFCE
:103D3000EAFFE850EF16020EE66EE66ADECFE6FF17
:103D4000DDCFE6FF050EE66EE66A6AEC2DF0326E18
:103D5000060EE15E325007D03B0EDECFE9FFDDCF2D
:103D6000EAFFE850EF16030EE15C02E2E16AE55279
:103D7000E16EE552E7CFD9FF1200000196514DE107
:103D8000010E966F975149E1010E976F020E785D13
:103D90000DE16FC0E9FF70C0EAFFEE52EF6A6FC03D
:103DA000E9FF70C0EAFFC80EEF6E1200780535E13A
:103DB0008B6B63C0E9FF64C0EAFFEE52400EEF6E0A
:103DC00063C0E9FF64C0EAFF020EE926000EEA22A2
:103DD000400EEE6E040EED6E63C0E9FF64C0EAFFB4
:103DE000840EEF6E010E8B6F65C0E9FF66C0EAFFBF
:103DF000EE52400EEF6E65C0E9FF66C0EAFF020EAC
:103E0000E926000EEA22400EEE6E040EED6E65C04D
:103E1000E9FF66C0EAFF800EEF6E12000001986BAA
:103E2000996B020E785D18E165C0E9FF66C0EAFF94
:103E3000EE52400EEF6E65C0E9FF66C0EAFF020E6B
:103E4000E926000EEA22480EEE6E040EED6E65C005
:103E5000E9FF66C0EAFF1DD07C510401465D000108
:103E60007D510401475904E246C47CF047C47DF00B
:103E70002BD96FC0E9FF70C0EAFF020EE926000EE1
:103E8000EA22480EEE6E040EED6E6FC0E9FF70C0C0
:103E9000EAFFC80EEF6E1200800E0401405D58E18B
:103EA0000001C00E7B6F04014351030A2FE0010A99
:103EB00009E0030A4BE10001BE0E796F5D0E7A6FD7
:103EC000120E3ED04251F66EF76AD890F636F736AB
:103ED000370EF6265E0EF7220900F5CF79F00A00BC
:103EE000F5CF7AF0020E0001F76A7925F66E7A5165
:103EF000F7220800F5CF7CF0030EF76A7925F66EFD
:103F00007A51F7220800F5CF7DF01200030E425DD2
:103F10001AE24251F66EF76AD890F636F736390E45
:103F2000F6265E0EF7220900F5CF79F00A00F5CFEC
:103F30007AF079C0F6FF7AC0F7FF0800F55000016B
:103F40007C6F7D6B120000017B6B120000017B6BAC
:103F50001200D9CFE6FFE1CFD9FF020EE12604011E
:103F6000486B496B40511F0B020A11E0030A0CE039
:103F7000010A35E100017B8F0401488100018705BA
:103F80002EE1040148832BD000017B8F28D0000153
:103F90007B8F040144BF0BD044510F0BE96EEA6ADA
:103FA000D890E936EA36670EE926000E0AD0445169
:103FB0000F0BE96EEA6AD890E936EA366F0EE92609
:103FC000000EEA22EECFDEFFEDCFDDFFDECFE9FF10
:103FD000DDCFEAFFEF50040B02E0010E486F000155
:103FE0007BAF07D0480E796F040E7A6F7B81020E8B
:103FF0007C6F020EE15C02E2E16AE552E16EE5529D
:10400000E7CFD9FF12006D9800017BBF2BD080AFA6
:1040100009D0020E786F995101E100DF0001976B22
:10402000966B120065C0E9FF66C0EAFFEE52400ED3
:10403000EF6E65C0E9FF66C0EAFF020EE926000EDA
:10404000EA22400EEE6E040EED6E65C0E9FF66C01A
:10405000EAFF8C0EEF6E6FC0E9FF70C0EAFF840EBE
:10406000EF6E1200040140AF0DD00001010E786F19
:10407000985101E1D3DE0001976B966B955123E1D6
:10408000BDEF1EF00001020E786F65C0E9FF66C04B
:10409000EAFFEE52400EEF6E65C0E9FF66C0EAFF30
:1040A000020EE926000EEA22400EEE6E040EED6EC0
:1040B00065C0E9FF66C0EAFF840EEF6E976B966BF2
:1040C000955101E15ADE1200D9CFE6FFE1CFD9FFC9
:1040D000E652400EDF6E00017C5D000E7D590AE263
:1040E0007CC0DFFF775102E1010E03D0770502E1CA
:1040F000020E776FDF50336AE8507C5D7C6F33507F
:104100007D597D6F6FC0E9FF70C0EAFFEE52DFCFCF
:10411000EFFF480E856F040E866F7BB118D0DF501D
:104120002DE079C0F6FF7AC0F7FF792B000E7A23D5
:104130000800F550E66E85C0E9FF86C0EAFF852BD2
:10414000000E8623E552E750EF6EDF06E8D7DF501A
:1041500015E079C0E9FF7AC0EAFF792B000E7A23D7
:10416000EF50E66E85C0E9FF86C0EAFF852B000EA2
:104170008623E552E750EF6EDF06E9D7E552E552B8
:10418000E7CFD9FF1200D9CFE6FFE1CFD9FF020E6A
:10419000E12663C0E9FF64C0EAFFEE52EFCFDFFF24
:1041A000DFCF32F032500001815D000E825902E211
:1041B00081C0DFFFDF50326E336AE850815D816F6E
:1041C00033508259826F010EDB6ADF50F36E010EAD
:1041D000DBCFF4FFF350F45C16E2010EDB50EA6A29
:1041E000480FE96E040EEA22EF50E66E7EC0E9FF4A
:1041F0007FC0EAFF7E2B000E7F23E552E750EF6E73
:10420000010EDB2AE2D7000ED8808155000E8255C0
:1042100027E265C0E9FF66C0EAFFEE52400EEF6E8E
:1042200065C0E9FF66C0EAFF020EE926000EEA2239
:10423000480EEE6E040EED6E63C0E9FF64C0EAFF47
:10424000EF50400B06E165C0E9FF66C0EAFFC80E0B
:1042500005D065C0E9FF66C0EAFF880EEF6E28D082
:1042600065C0E9FF66C0EAFFEE52400EEF6E65C022
:10427000E9FF66C0EAFF020EE926000EEA22400EC0
:10428000EE6E040EED6E65C0E9FF66C0EAFF840EB7
:10429000EF6E8351841107E005D084C0FAFF00015E
:1042A0008351F96EFADF0001809F955101E165DDD0
:1042B000020EE15C02E2E16AE552E16EE552E7CF0F
:1042C000D9FF1200D9CFE6FFE1CFD9FFE6520001B6
:1042D0007B8F030EE66EE66AE66A710EE66E0F0EDF
:1042E000E66E04EC2EF0326E050EE15E3250DF6AAF
:1042F000DF50326E336A100E325C000E335810E21B
:10430000DF50040DF3CFE9FFF4CFEAFF000EE926FA
:10431000040EEA22EE6AEE6AEE6AEE6ADF2AE8D757
:104320006D8C010EE66EE66AE66A620EE66E000EBF
:10433000E66E04EC2EF0326E050EE15E32506D9C9E
:104340000001080E6F6F040E706F000E636F040E95
:10435000646F63C065F0666F42C461F0615102E151
:10436000100E12D0010EE66EE66A610EE66E000EC9
:10437000E66E010EE66EE66A6AEC2DF0326E060E0F
:10438000E15E32500001200E606FE552E552E7CF4A
:10439000D9FF1200D9CFE6FFE1CFD9FF020EE12607
:1043A000000EDE6E040EDD6EFD0EDB50E824346E72
:1043B000FE0EDB50040DF3503424040DF4CF33F023
:1043C000D9CFE9FFDACFEAFFF350EE263350ED22E2
:1043D000DECFE9FFDDCFEAFFEF9EFD0EDB500AE105
:1043E000FE0EEA6ADB34FE0BEA36E96E670EE9265A
:1043F000000E09D0FE0EEA6ADB34FE0BEA36E96EE7
:104400006F0EE926000EEA22DECFEEFFDDCFEDFFD4
:10441000DECFE9FFDDCFEAFFEF9CDECFE9FFDDCFA6
:10442000EAFF040EE926000EEA22EF8C020EE15CA0
:1044300002E2E16AE552E16EE552E7CFD9FF1200F0
:10444000D9CFE6FFE1CFD9FF020EE126FD0EDBA4B6
:1044500007D0E66AFE0EDBCFE6FF9CDFE552E552B1
:10446000FD0EDBA208D0010EE66EFE0EDBCFE6FFEE
:1044700091DFE552E552FE0EDB50336A700F326E6B
:104480000F0E332232C0DEFF33C0DDFFDECFE9FF87
:10449000DDCFEAFFFD0EDBCFEFFF020EE15C02E2B3
:1044A000E16AE552E16EE552E7CFD9FF1200D9CFBC
:1044B000E6FFE1CFD9FF020EE126FE0EDB5020E140
:1044C00065C0E9FF66C0EAFFEE52400EEF6E65C0C0
:1044D000E9FF66C0EAFF020EE926000EEA22400E5E
:1044E000EE6E040EED6E65C0E9FF66C0EAFF8C0E4D
:1044F000EF6E6FC0E9FF70C0EAFF840EEF6E3BD035
:10450000FD0EDB50E824346EFE0EDB50040DF3503C
:104510003424040DF3CF32F0F4CF33F0000E322602
:10452000040E332232C0DEFF33C0DDFF840EDECF47
:10453000E9FFDDCFEAFFE850EF12FD0EDB50E82483
:10454000346EFE0EDB50040DF3503424010F040DC5
:10455000F3CF32F0F4CF33F0000E3226040E3322C4
:1045600032C0DEFF33C0DDFF840EDECFE9FFDDCFDA
:10457000EAFFE850EF12020EE15C02E2E16AE55266
:10458000E16EE552E7CFD9FF1200D9CFE6FFE1CFC8
:10459000D9FF020EE126FD0EDB500AE0FE0EEA6AAC
:1045A000DB34FE0BEA36E96E6F0EE926000E09D009
:1045B000FE0EEA6ADB34FE0BEA36E96E670EE92688
:1045C000000EEA22EECFDEFFEDCFDDFFD9CFE9FF0F
:1045D000DACFEAFFEE50ED1003E1F36AF46A44D05B
:1045E000DECFE9FFDDCFEAFF020EE926000EEA2268
:1045F000FB0EDBCFEEFFFC0EDBCFEDFFDECFE9FFE6
:10460000DDCFEAFFEE52FA0EDBCFEFFF400EDECF3A
:10461000E9FFDDCFEAFFE850EF16880EDECFE9FFB5
:10462000DDCFEAFFE850EF12FD0EDB500AE0FE0E90
:10463000EA6ADB34FE0BEA36E96E6F0EE926000EFD
:1046400009D0FE0EEA6ADB34FE0BEA36E96E670E2D
:10465000E926000EEA22EF74DECF32F0DDCF33F030
:1046600032C0F3FF33C0F4FF020EE15C02E2E16A04
:10467000E552E16EE552E7CFD9FF1200D9CFE6FF50
:10468000E1CFD9FF6DA84ED0FE0EEA6ADB34FE0BF7
:10469000EA36E96E6F0EE926000EEA22EE50EFCF01
:1046A000EAFFE96E400EEE16EE6AEE6AEE6AFE0E64
:1046B000EA6ADB34FE0BEA36E96E6F0EE926000E7D
:1046C000EA22EE50EFCFEAFFE96EEE7CFE0EEA6AD8
:1046D000DB34FE0BEA36E96E6F0EE926000EEA22A5
:1046E000EF74400E326EFE0EEA6ADB34FE0BEA36E1
:1046F000E96E6F0EE926000EEA22EE50EFCFEAFFD8
:10470000E96E3250EF16FE0EEA6ADB34FE0BEA3633
:10471000E96E6F0EE926000EEA22EE50EFCFEAFFB7
:10472000E96EEF7CE552E7CFD9FF12006D6A696A46
:104730000001606B12000001605113E16D6A696A4B
:10474000160E6F6E9F0E6B6E7B0E696ED08EA29AE8
:10475000A08AF28E6DB602D06D86FCD70001010EE4
:04476000606F120074
:0C476400EEEC28F0FB0EDBCFF3FFDB06D1
:10477000F35000090AE03CEC29F0FA0EA7EC29F00E
:10478000F3E1331CF1E1010E01D0000E1DEF29F021
:10479000EEEC28F03B0EE12402E3E168E652E16E24
:1047A000010EDB6A020EDB6AF90EDBCFF6FFFA0EB2
:1047B000DBCFF7FFFB0EDBCFF8FF0800F550DF6E15
:1047C000DF5002E141EF28F0250EDF5C02E034EF1C
:1047D00028F0030EDB6A040EDB6A050EDB6A060EA8
:1047E000DB6A070EDB6A56EC28F02D0EDF5C0CE06E
:1047F0002B0EDF5C09E0200EDF5C06E0230EDF5CA1
:1048000003E0300EDF5C1AE1DF50300A14E0130AD7
:104810000FE0030A0AE00B0A05E0060AE4E1030ED2
:10482000DB80E1D7030EDB82DED7030EDB84DBD730
:10483000030EDB86D8D7030EDB88D5D72A0EDF5CC4
:104840001BE152EC28F0A0EC28F010E0030EDB8016
:1048500026682768130EDBCF2BF0140EDBCF2CF06D
:1048600017EC2DF0040E24C0DBFF03D0130E89ECEF
:1048700028F056EC28F00BD0090EDB6AF7EC28F094
:1048800003E06BEC29F0FAD7090E89EC28F0030E4F
:10489000DBB0DB982E0EDF5C1BE156EC28F02A0E15
:1048A000DF5C0BE152EC28F0A0EC28F003E1130EE2
:1048B000DBEC28F056EC28F00BD0090EDB6AF7ECA5
:1048C00028F003E06BEC29F0FAD7090EDBEC28F0B6
:1048D000680EDF5C07E156EC28F0680EDF5C1DE136
:1048E000030E18D0740EDF5C17E07A0EDF5C14E064
:1048F000480EDF5C06E0540EDF5C03E05A0EDF5C1E
:1049000002E1020E07D06C0EDF5C03E06A0EDF5C92
:1049100004E1010E2EEC29F0C9DBDF506E0A01E143
:104920007FD31E0A01E192D1200A01E18FD13F0A13
:1049300001E149D11A0A01E146D10D0A01E143D151
:10494000200A01E140D13A0A01E13DD1200A01E10A
:104950003AD1260A01E135D10D0A01E132D11A0A14
:1049600001E1D9D0200A4AE0300A1FE0460A0EE0F1
:10497000250A01E083D3D950F90FE96EFF0EDA2042
:10498000EA6E010EEE5E000EEE5AEE5A3CEC29F095
:10499000250EE66E95DB03E1331C01E169D338ECAB
:1049A00029F001E26BD3DB2A69D3080EDB6A040E1F
:1049B000DB50010806E2040EDB0400EC29F0DB50BA
:1049C0008BDB080EDB5009E0030EDB50010B05E129
:1049D00072DB01E04DD3080EDB6A64DBEFCFDFFF53
:1049E000B0EC29F003E1331C01E142D338EC29F0AB
:1049F00001E3DB2A60DB01E141D33AD3070EDB5050
:104A000002080FE17CEC29F0030E43EC29F00E0EB6
:104A1000EECFDBFF0F0EEECFDBFF100EEECFDBFF96
:104A200020D0F70EDBCF35F0F80EDBCF36F0020EDC
:104A3000355E000E365AF70E35C0DBFFF80E36C075
:104A4000DBFF35C0E9FF36C0EAFF33EC29F0346AFA
:104A50000E0E32C0DBFF0F0E33C0DBFF100E34C072
:104A6000DBFF0E0EDBCFE6FF0F0EDBCFE6FF100EF7
:104A7000DBCFE6FF2CEC2EF0E552E552E552130EAB
:104A800025C0DBFF140E26C0DBFF060EDB5005E061
:104A9000130E77EC29F001E26ADB9BEC29F002E2CD
:104AA000130E37DB5EEC29F006E0040E77EC29F0FC
:104AB00002E2050E2EDB030EDBB005D0FCDA01E0CE
:104AC000D7D2080EDB6A090EDB6A0E0EDBCFF6FFCB
:104AD0000F0EDBCFF7FF100EDBCFF8FF0800F5500D
:104AE000DF6EDF5014E0A1EC29F011E2B0EC29F008
:104AF00003E1331C01E1BCD2BBDB01E3DB2A090E7D
:104B0000DB2AD9500E0FE96E000ECBDBE7D7D3DAE4
:104B100001E1B4D2ADD2C6DA110EEECFDBFF120E38
:104B2000EDCFDBFF110EDBCFE6FF120EDBCFE6FF92
:104B30001EEC2EF0E552E552130EF3CFDBFF140E00
:104B4000F4CFDBFF060EDB5004E0130ED0DB01E2F6
:104B50000EDB9BEC29F002E2130EDBDAAFDB05E0A3
:104B6000040EC5DB02E2050ED4DA030EDBB005D07D
:104B7000A2DA01E07DD2080EDB6A090EDB6A110EB3
:104B8000DBCFE9FF120EDBCFEAFFEFCFDFFFDF5015
:104B900014E0D7DB12E2E4DB03E1331C01E168D26D
:104BA00067DB01E3DB2A090EDB2A110EDB2ADBCFF0
:104BB000E9FF120EE8E3DB2AE6D77DDA01E15ED2F7
:104BC00057D2030EDB8E070EDB0410E195DB040EDB
:104BD0005ADB0A0EEECFDBFF0B0EEECFDBFF0C0E27
:104BE000EECFDBFF0D0EEECFDBFF6CD0070EDB5000
:104BF00003082CE1030EDBAE0DD0B2DA020E76DA3A
:104C0000EFCF32F0336A346A356A32AE39D0336866
:104C1000346835D0F70EDBCF33F0F80EDBCF34F04D
:104C2000020E335E000E345AF70E33C0DBFFF80E6F
:104C300034C0DBFF33C0E9FF34C0EAFFEFCF32F00E
:104C40000A0E32C0DBFF0B0EDB6A38D0070EDB50DA
:104C5000020809E1030EDBAE04D059DB34AE10D0FC
:104C60000ED055DB0DD0030EDBAE12D079DA020E7A
:104C70003DDAF9DA346A356A33AE02D03468356821
:104C8000E2DA0C0E34C0DBFF0D0E35C0DBFF1AD0AC
:104C9000F70EDBCF34F0F80EDBCF35F0020E345ECA
:104CA000000E355AF70E34C0DBFFF80E35C0DBFFBF
:104CB00034C0E9FF35C0EAFFD6DAC5DA0C0EDB6A8C
:104CC0000D0EDB6A060EDB5005E1010EF36E050EDC
:104CD000F3CFDBFF150EDB6A160EDB6AD950370FF8
:104CE000326E000EDA20336E390E32C0DBFF3A0E20
:104CF00033C0DBFF380EDB6A080EDB6A0A0EAEDA61
:104D0000DF50780A12E0200A10E0280A0CE0200A9E
:104D10000AE03F0A06E00D0A02E0200A08E1020E5E
:104D200005D0080E03D0080EDF26100E97DA030E0A
:104D3000DBBE02D0DB92DB94DB50800B24E08ADA0E
:104D4000D890030EEB50000A08E6000EEE5C000E51
:104D5000EE58000EEE58000EEE5815E213DA2968F0
:104D60002A682B682C6820EC2FF00A0E20C0DBFF8D
:104D70000B0E21C0DBFF0C0E22C0DBFF0D0E23C08B
:104D8000DBFF2D0E08D0030EDBA202D02B0E03D0CA
:104D9000DBA408D0200EF36E170EF3CFDBFF150E49
:104DA000DB2A02D0170EDB6A050EDB5003E1B7D910
:104DB00001E189D0D40E326E5F0E336E000E346E78
:104DC000070EDBCF35F0366A376A386A35C029F00E
:104DD00036C02AF037C02BF038C02CF0D3D97EEC87
:104DE0002FF032502024F36E33502120F46E3450D3
:104DF0002220F86EF4CFF7FFF3CFF6FF0800090E7C
:104E0000F5CFDBFF580EDF5C0FE1610EF36E090E8C
:104E10007BD90AE3200E326E090EDBCFE7FF32505A
:104E2000E75E090EE7CFDBFF070EDBCF32F0336A18
:104E3000346A356A0FDA32C029F033C02AF034C040
:104E40002BF035C02CF0EECF24F0EECF25F0EECFD6
:104E500026F0EFCF27F07EEC2FF027C0EDFF26C025
:104E6000EDFF25C0EDFF24C0EFFF390EDBCFE9FFDA
:104E7000DB063A0EDBCFEAFF01E2DB06090EDBCFF1
:104E8000EFFF150EDB2A4BD995E1030EDBA61DD0F3
:104E90006F0EDF5C06E1C1D918E3150EDB285BDA83
:104EA00014D0780EDF5C09E0580EDF5C06E0620E7D
:104EB000DF5C03E0420EDF5C08E1020EF36E160ECB
:104EC000F3CFDBFF02D0150EDB6A030EDB50100BB5
:104ED0000EE0040EDBCF32F0050EDB50D8803254EA
:104EE00006E2060EDB5003E1040EDB5034DA95D9FE
:104EF0000AE2050EDBCFE7FF150EDB50E75E050E7D
:104F0000E7CFDBFF02D0050EDB6A040EDBCF32F009
:104F1000160E45D9D880325414E2160EDBCFE6FFC8
:104F2000150EDBCFE6FF040EDBCFE6FF050EDB50F0
:104F3000E552E75CE552D880E754E552D880E75463
:104F40005FD9030EDB50010B0BE1080EDB5008E0CC
:104F5000B2D801E08DD0080EDB50BED8080EDB6A57
:104F6000170EDB5007E088D9170EF1D903E1331C87
:104F700001E17ED0160EDB5016E07ED9300EE66ED3
:104F80009FD802E1331C74E077D9DFCFE6FF9DECB8
:104F90002EF0E552E552E552F4CF33F00001F31C58
:104FA00002E1331C65E0050EDBCF32F0160EDB505C
:104FB000D880325409E2050EDBCFE7FF160EDB5036
:104FC000E75E050EE7CFDBFF300EE66E050ECBD9B0
:104FD0004FE1390EDB2ADBCFE9FF3A0E01E3DB2A92
:104FE000DBCFEAFF090EEFCFDBFFDB500EE044D949
:104FF000090EADD902E1331C3BE0390EDB2ADBCFD1
:10500000E9FF3A0EEDE3DB2AEBD755D831E1160E76
:10501000DBCFE6FF080EC3D8E552E7245DD82ED0DB
:10502000070EDB50030A1CE0010A14E0030A07E044
:105030007BD9DBCFEEFF020EDBCFEDFF1FD0F5D823
:10504000376A35AE02D0366837682CD8BCD837C03E
:10505000EEFF14D0EAD835BE366824D8B4D80ED0C6
:1050600063D9DBCFEFFF0AD07BD905E1331C03E125
:10507000F368F46810D0FCD801E3DB2A79D9DDEFBE
:1050800023F0010EDBCF32F0020EDBCF33F032C063
:10509000F3FF33C0F4FF3B0EE15C02E2E16AE5524C
:1050A000E16ECBD029D9020E43EF29F061D9080077
:1050B000F550DF6E1200200EE66E080EB3EF29F0F9
:1050C0009DEC2EF0E552E552E552F3CF32F0F4CFED
:1050D00033F00001F31C1200326E336AD950010F15
:1050E0004DD93250EE263350ED221200365E000EBE
:1050F000375AF70E36C0DBFFF80E37C0DBFF36C07D
:10510000E9FF37C0EAFF1200DBCFF4FFF350F45C95
:105110001200DB50E76E040EE7CFDBFF12000A0E31
:10512000DBCF32F00B0EDBCF33F00C0EDBCF34F0E5
:105130000D0EDBCF35F03250331034103510120025
:10514000130EEECFDBFF140EEDCFDBFF130EDBCF24
:1051500032F0140EDBCF33F00001800E3314120056
:10516000F70EDBCF36F0F80EDBCF37F01200050E6E
:10517000DB50E66ED950130F01D9E552E750EE6EC1
:10518000ED6A12000A0EDBCF24F00B0EDBCF25F008
:105190000C0EDBCF26F00D0EDBCF27F01200DBCF9D
:1051A000E6FF150EDBCFE6FF050EDB50E552E724E8
:1051B000E552E7241200DB50CED8010EF36E060E46
:1051C000F3CFDBFF1200EE50EFCFEAFFE96E34C001
:1051D000EEFF35C0EEFF36C0EEFF1200D9CFE6FF7E
:1051E000DACFE6FFE1CFD9FFE2CFDAFF1200DFCF5F
:1051F000E6FFE66A6CEC2FF0E552E552F350120040
:10520000E76E080EE7CFDBFF1200EECF32F0EECFF5
:1052100033F0EFCF34F0356A1200050EDBCF32F0F9
:10522000150EDB50D88032541200010EDBCF34F063
:10523000020EDBCF35F0366A1200E552E5CFDAFF19
:10524000E7CFD9FF12000A0E32C0DBFF0B0E33C0CE
:10525000DBFF1200D9500A0FBEEF29F0F36E070EE4
:10526000F3CFDBFF1200EECF32F0EFCF33F01200BE
:10527000010EDB2A020E1200FC0EDBCFE6FFFD0E54
:10528000DBCFE6FF1200325E000E335AF70E32C05B
:10529000DBFFF80E33C0DBFF32C0E9FF33C0EAFFAB
:1052A0001200DA20EA6EEF2AEECFF6FF000EEF22B0
:1052B000EECFF7FFEF22EECFF8FF1200040EDBCFA8
:1052C000E6FF130EDB50E552E75C9ADFDB5004DFAC
:1052D000060EDB501200090EDB500A0DF350DF24DE
:1052E000D00FE76E090EE7CFDBFF56EF28F0DB505B
:1052F000F36E050E84EF28F0F70EDBCF32F0F80ED8
:10530000DBCF33F01200DFCFE6FF60EF28F028DFBD
:10531000030EECDE05EF29F0B2EC23F0E552E55286
:10532000E552E55200091200BDDEEE50EFCFEAFF74
:10533000E96E010E1200130EDB50F36E040E84EFC3
:1053400028F0040EDB50F36E090E84EF28F0DBCF5B
:10535000E6FF60EF28F0E76E050EE7CFDBFF1200F7
:105360008BDF83EF29F0DBCFE6FF86DF8CEF29F0C0
:10537000D950F90FE96EFF0E51EF29F0E96E000EDA
:06538000DA20EA6E1200C3
:0A538600040140511F0B010801E073
:1053900012004051600BE842E842E842E842E8422D
:1053A000010801E01200445103E0440501E012004D
:1053B0004151220A31E0030A24E0010A15E0210AE2
:1053C0000DE0010A01E012000001E20E796F020E09
:1053D0007A6F080E7C6F7D6B7B8121D00001E20E1D
:1053E000796F020E7A6F1BD046C481F047C482F0F9
:1053F0000001880E7E6F050E7F6F836B846B808F3C
:1054000012000001880E796F050E7A6F070E7C6F0F
:105410007D6BC10E7B6F120042C4DDF200017B8FF9
:1054200012000501886B4B0E896F8A6B8B6B8C6B3E
:105430008D6B080E8E6F0201D16B1A0EE66E020E96
:10544000E66E20EC22F0E552E5521E0EE66E030EEB
:10545000E66E20EC22F0E552E552400EE66E080EB4
:10546000E66E050EE66EE66A030EE66EC5EC22F009
:10547000326E050EE15E3250F3CFD9F2F4CFDAF29C
:105480000201DB6BDC6BD26B1200D9CFE6FFE1CF00
:10549000D9FF0201D16BD951DA1102E1000E08D017
:1054A000D9C2E9FFDAC2EAFFEF50800B01E0010E3A
:1054B000000945E1FC0EDBCF32F0D9C2E9FFDAC2C8
:1054C000EAFFEE52EF50D880325408E2D9C2E9FF29
:1054D000DAC2EAFFEE52FC0EEFCFDBFFD16BFC0E1F
:1054E000DB50D15D19E2D151EA6A080FE96E050E71
:1054F000EA22EF50E66ED151E76EFD0EDBCFE9FFF9
:10550000FE0EDBCFEAFFE750E926000EEA22E55265
:10551000E750EF6ED12BE3D7400EE66E080EE66E35
:10552000050EE66EE66A030EE66EC5EC22F0326EFC
:10553000050EE15E3250F3CFD9F2F4CFDAF2020178
:10554000D151E552E7CFD9FF1200D9CFE6FFE1CF25
:10555000D9FFA09A0201D2510CE1FD0EDBCFD3F2AC
:10556000FE0EDBCFD4F2FC0EDBCFD7F2010ED86FEC
:10557000D26FA08AE552E7CFD9FF1200D9CFE6FF5C
:10558000E1CFD9FF030EE126A09A0201D2512DE10D
:10559000DF6AFD0EDBCF26F0FE0EDBCF27F0DE52FA
:1055A00026C0DEFF27C0DDFFDD52DF2ADF50326E6E
:1055B000336AFF0E321802E133500BE0010EDBCFED
:1055C000E9FFDB2A020EDBCFEAFF01E3DB2AEF5023
:1055D000ECE1FD0EDBCFD3F2FE0EDBCFD4F2DFCF5A
:1055E000D7F20201010ED86FD26FA08A030EE15CE0
:1055F00002E2E16AE552E16EE552E7CFD9FF12001F
:10560000D9CFE6FFE1CFD9FF030EE126A09A020130
:10561000D2512EE1DF6AFD0EDBCF26F0FE0EDBCF8E
:1056200027F0DE5226C0DEFF27C0DDFFDD52DF2A75
:10563000DF50326E336AFF0E321802E133500CE055
:10564000010EDBCFF6FFDB2A020EDBCFF7FF01E313
:10565000DB2A0800F550EBE1FD0EDBCFD3F2FE0EA6
:10566000DBCFD4F2DFCFD7F20201D86B010ED26FBD
:10567000A08A030EE15C02E2E16AE552E16EE552C6
:10568000E7CFD9FF1200D9CFE6FFE1CFD9FF020E55
:10569000E126A09A0201DB51DC1102E1000E08D0E4
:1056A000DBC2E9FFDCC2EAFFEF50800B01E0010E34
:1056B000000906E1030ED25D01E1D26BD25102E195
:1056C000A08A7ED0020ED25D16E1E66A000EE66E7A
:1056D000E66A010EE66E030EE66EC5EC22F0326E4F
:1056E000050EE15E3250F3CFDBF2F4CFDCF20201C3
:1056F000030ED26F64D0D20562E1400E326E336A7F
:10570000D751325C000E335803E2400EDF6E02D0F8
:10571000D7C2DFFFDF50D75DD76F480ED56F050EBC
:10572000D66F010EDFCFDBFFD85116E1010EDB5043
:1057300028E0D3C2F6FFD4C2F7FF0800F550D5C267
:10574000E9FFD6C2EAFFEF6ED52B000ED623D32B8E
:10575000D423010EDB06EAD7010EDB5012E0D3C2E0
:10576000E9FFD4C2EAFFEF50D5C2E9FFD6C2EAFF93
:10577000EF6ED52B000ED623D32BD423010EDB06E0
:10578000EBD70201D75107E1400EDF5C02E1020EC8
:1057900001D0030ED26FDFCFE6FF480EE66E050E96
:1057A000E66E010EE66E030EE66EC5EC22F0326E7A
:1057B000050EE15E3250F3CFDBF2F4CFDCF2A08ACB
:1057C000020EE15C02E2E16AE552E16EE552E7CFEA
:0457D000D9FF1200EB
:0C57D4005374617475733D25690D0A0063
:1057E0002135204572723A204E65656420636F6DE5
:1057F0006D61206E6578742C20666F756E643A203A
:10580000272563270D0A0050492C2531750D0A0004
:105810004D522C253033750D0A002C25303475007F
:105820004100492C253033692C253033692C253033
:1058300033692C253033692C253033690D0A00215A
:1058400038204572723A20556E6B6E6F776E20630A
:105850006F6D6D616E642027256325633A2532588C
:10586000253258270D0A002138204572723A2055FA
:105870006E6B6E6F776E20636F6D6D616E64202747
:1058800025633A253258270D0A00213720457272C8
:105890003A204578747261207061726D617465722E
:1058A0000D0A002136204572723A20496E76616CED
:1058B000696420706172616D7465722076616C75C7
:1058C000650D0A002134204572723A204D697373C8
:1058D000696E6720706172616D65746572287329E5
:1058E0000D0A002133204572723A20525820427529
:1058F00066666572206F76657272756E0D0A00219C
:1059000032204572723A205458204275666665729C
:10591000206F76657272756E0D0A002130200D0AB7
:10592000002008002573001B5B421B5B314B1B5B97
:03593000304700FD
:0C5934001E6AE86A2CAEA7EF2CF0296C6C
:105940002A1E2B1E2C1E2A222B222C221E1E27AE84
:10595000B2EF2CF0246C251E261E271E252226229F
:1059600027221E1E7EEC2FF027BEC9EF2CF01EAEA4
:10597000000C246C251E261E271EE86A25222622DE
:105980002722206C211E221E231E212222222322B6
:10599000000C1EBEB9EF2CF01F88FF0C27C031F0A1
:1059A00026C030F025C02FF025502A02F4CF23F076
:1059B000F3CF22F026502B02F4CF25F0F3CF24F0C2
:1059C0002A02F3502326F4502422E86A25222F507D
:1059D0002B02F3502326F4502422E86A2522275074
:1059E0002A02F3502426F450252227502B02266A3F
:1059F000E86A2622F3502526F45026222F502C0246
:105A0000F3502426F4502522276AE86A262227220A
:105A100030502C02F3502526F4502622E86A272223
:105A200031502C02F3502626F4502722000C27C0B8
:105A300031F026C030F026502B02F4CF25F0F3CF02
:105A400024F027502C02F4CF27F0F3CF26F02B02BE
:105A5000F3502526F4502622E86A272230502C02E3
:105A6000F3502526F4502622E86A27222CAE3DEF7B
:105A70002DF03050265E3150275A31AE000C2B509D
:085A8000265E2C50275A000C91
:085A880008D80001605102E1A1
:105A90009BEC23F0F3EC06F0F8D70F0EC1122CECC0
:105AA00006F0AAEF1AF01200120012001200C3EF63
:105AB00029F0120011EF2AF06D840101080EF56F34
:105AC000070EF66FF507000EF65BF551F611FAE1D9
:105AD0006D941200D9CFE6FFE1CFD9FFFD0EDBCFE9
:105AE00026F0FE0EDBCF27F0720E261801E12750BC
:105AF00033E0E868261802E17F0E27182BE0740EC9
:105B0000261801E1275024E0750E261801E12750E0
:105B10001DE0730E261801E1275016E0030E26182B
:105B200001E127500FE0020E261801E1275008E09E
:105B3000010E261801E1275001E010D0BBDF0FD085
:105B4000B8DF0DD0B4DF0BD0B0DF09D0ACDF07D0A9
:105B5000ABDF05D0ABDF03D0000001D000D0010ED9
:0A5B600000D0E552E7CFD9FF120094
:065B6A001E0EF66E080E8F
:105B7000F76E000EF86E01010900F550F06F090094
:105B8000F550F16F03E1F06701D03DD00900F55009
:105B9000EB6F0900F550EC6F0900F550ED6F09004F
:105BA0000900F550E96E0900F550EA6E0900090098
:105BB0000900F550EE6F0900F550EF6F090009007C
:105BC000F6CFF2F1F7CFF3F1F8CFF4F1EBC1F6FF36
:105BD000ECC1F7FFEDC1F8FF0101EE5302E1EF5315
:105BE00007E00900F550EE6EEE07F8E2EF07F9D78F
:105BF000F2C1F6FFF3C1F7FFF4C1F8FF0101F007AE
:085C0000000EF15BBFD712009A
:085C0800FE0EE3CFE9FFFF0EE1
:105C1000E3CFEAFFE9CFF3FFEACFF4FFFB0EE35057
:105C200003E1FC0EE35009E0FB0EE30602E2FC0E8A
:105C3000E306FD0EE350EE6EF1D71200FE0EE3CF49
:105C4000E9FFFF0EE3CFEAFFF36AF46AEE5203E0E6
:105C5000F34AF42AFBD71200FF0EE3CFF8FFE55218
:105C6000FF0EE3CFF7FFE552FF0EE3CFF6FFE5525D
:105C7000E66AE66AE66A0900F55209E0FD0EE32AE3
:105C800005E1FE0EE32A02E1FF0EE32AF4D7FD0E42
:105C9000E3CF25F0FE0EE3CF26F0FF0EE3CF27F093
:025CA0001200F0
:0E5CA200D9CFE6FFDACFE6FFE1CFD9FFE2CFA0
:105CB000DAFFE652E652E652E652D950FB0F326E58
:105CC000FF0EDA20336E32C0DEFFDD6EDECFE6FF80
:105CD000DDCFE6FFFB0EDBCFE6FFFC0EDBCFE6FF02
:105CE000FD0EDBCFE6FFF7C1E6FFF8C1E6FFC8EC2B
:105CF00023F0326E070EE15C02E2E16AE552E16EEA
:105D00003250020EF3CFDBFF030EF4CFDBFF020EA7
:105D1000DBCF32F0030EDBCF33F032C0F3FF33C002
:105D2000F4FF040EE15C02E2E16AE552E16EE55245
:0A5D3000E5CFDAFFE7CFD9FF12003C
:065D3A00D9CFE6FFDACF2D
:105D4000E6FFE1CFD9FFE2CFDAFFFB0EDBCF32F087
:105D5000FC0EDBCF33F00001800E33141AE1FB0E92
:105D6000DBCFE9FFFC0EDBCFEAFFEECFF3FFEDCF99
:105D7000F4FFEE2A000EEF22F3CFE9FFF4CFEAFFA3
:105D8000FD0EDBCFEFFFEF50336AF36E33C0F4FF4D
:105D900010D0FB0EDB50FE0806E1FD0EDBCFE6FF68
:105DA000D1EC2FF005D0FD0EDBCFE6FF19EC09F0AA
:0E5DB000E552E552E5CFDAFFE7CFD9FF12004A
:025DBE001201D0
:105DC000000202000040D80492FD8201010200019D
:105DD00009024300020100C032090400000102026E
:105DE000010005240010010424020205240600011C
:105DF00005240100010705820308000209040100CF
:105E0000020A0000000705030240000007058302A4
:105E10004000000403090418035300630068006D88
:105E20000061006C007A0048006100750073000892
:0F5E300003550042005700D05D135E175E2F5ED2
:105E400024502902F3CF20F0F4CF21F02A02F3509E
:105E50002126000EF420226E24502B02F35022261D
:105E6000000EF420236E24502C02F35023262550DC
:105E70002902F3502126F4502222000E232225501D
:105E80002A02F3502226F450232225502B02F350ED
:105E9000232626502902F3502226F450232226508E
:105EA0002A02F350232627502902F35023261200FA
:105EB000FF0EE124E96EFF0EE220EA6EEDCFF4FF63
:105EC000EFCFF3FFF46607D0600EF36404D07B0ECF
:105ED000F36001D0F39A1200F36AF46AFF0EE12432
:105EE000E96EFF0EE220EA6EED6607D02F0EEF643A
:0C5EF00004D03A0EEF6001D0F32A12003B
:045EFC00236A226A89
:105F0000216A206A200EE76ED89024362536263680
:105F1000273620362136223623362950205C2A5057
:105F200021582B5022582C50235809E32950205E29
:105F30002A50215A2B50225A2C50235A242AE72E19
:045F4000E4D7120090
:0C5F44004F4B0D0A000D0A00554257207B
:105F5000465720442056657273696F6E20312E3487
:055F60002E390D0A00BE
:0A5F6600000EF36E00EE00F0080ECE
:105F700001D81200EA6002D0EE6AFCD7F350E96063
:065F80001200EE6AFCD7DE
:0A5F860016EE00F026EE00F0F86AB7
:105F90001F9CB5EC2DF003EC04F044EC2DF0FBD786
:025FA0001200ED
:0E5FA200FF0EE350ACBA04D0AF6AAB8EAC8AEF
:0E5FB000949CACA2FED7AD6EF36EF46A1200A4
:025FBE00FF0ED4
:105FC000E350E84E1200000000D000D000D0E82ED0
:045FD000FAD71200EA
:0C5FD400303132333435363738396162F1
:055FE00063646566002A
:0B5FE5000000000000000000000000B1
:105FF00000000000000000000000000000000000A1
:106000000000000000000000000000000000000090
:106010000000000000000000000000000000000080
:106020000000000000000000000000000000000070
:076030000000000000000069
:00000001FF
